:10000000F89411240FEF0DBF00E10EBFA0E0B1E0A6
:10001000C2E8D1E0CA1BDB0B2196E0E9F8E02197AA
:1000200019F005900D92FBCFA2E8B1E0CEE8D1E047
:10003000CA1BDB0B2196219711F01D92FCCF02D039
:100040000C9402F0AF92BF92CF92DF92EF92FF92A8
:100050000F931F93CF93DF9380E091E00E94020300
:1000600082E191E00E94020380E391E00E9402039A
:100070000F2EF5E3AF2EBB24F02D0F2EF9E3EF2E5C
:10008000FF24F02D0F2EFBE3CF2EDD24F02D8FE08B
:1000900084BB1ABA00E010E08FE0F601808381E0B3
:1000A00090E0002E02C0880F991F0A94E2F7809515
:1000B0008F70F501808360E070E08AE090E00E943C
:1000C000CC00F701808199279C012F703070C0E02F
:1000D000D0E0C9010C2E02C0959587950A94E2F7ED
:1000E00080FF04C02196C430D1059CF3C430D105F3
:1000F00031F1F701808199270C2E02C095958795E3
:100100000A94E2F780FFF5CF8EE491E00E940203AB
:10011000C801880F991F880F991F835A9E4FFC01B1
:10012000EC0FFD1F80810E94E0028EE691E00E94AC
:10013000020360E070E08AE090E00E94CC000F5F74
:100140001F4F043011050CF4A7CFA4CFA09182015A
:10015000B0918301AB2BA9F4109290006FE069B9C4
:1001600052E05BB948E14AB936E0309395008F9A86
:1001700097988E98969A21E030E0309383012093EF
:1001800082015F9904C097985F9BFECF979A8CB1CC
:10019000992787FD909508952F923F924F925F92F5
:1001A0006F927F928F929F92AF92BF92CF92DF9287
:1001B000EF92FF920F931F93CF93DF93CDB7DEB7EC
:1001C0002A970FB6F894DEBF0FBECDBF8D839E83F6
:1001D0006F8378871FBC01E00EBD10927A004CB48B
:1001E00049823DB43A8229803A8060908A017090B9
:1001F0008B01261837083694279436942794369422
:1002000027944090880150908901420C531C5092D1
:100210008901409288014101AA24BB24D501C4016F
:10022000E3E0880F991FAA1FBB1FEA95D1F7881931
:100230009909AA09BB09680E791EC501B40120E419
:1002400030EB45E050E00E94E00380908401909004
:100250008501A0908601B0908701860E971EA81E8A
:10026000B91EC501B40120E432E44FE050E00E9421
:100270001204DA01C90129833A83620E731E709257
:100280008B0160928A01AA27BB27BC01CD0120E423
:1002900032E44FE050E00E94E003861A970AA80A71
:1002A000B90A8092840190928501A0928601B09251
:1002B000870112011FBC11E01EBD10927A00FCB430
:1002C000FB82DDB4DC822B813C812619370936950F
:1002D000279536952795369527957201E20EF31EE0
:1002E0002701E986FA8644275527DA01C90163E028
:1002F000880F991FAA1FBB1F6A95D1F7821B930B0A
:10030000A40BB50B8301080F191FCA01B90120E422
:1003100030EB45E050E00E94E0036B017C01C80C2B
:10032000D91CEA1CFB1CC701B60120E432E44FE0F3
:1003300050E00E941204DA01C9012B833C83020FB2
:10034000131F3801AA27BB27BC01CD0120E432E4EA
:100350004FE050E00E94E003C61AD70AE80AF90A03
:1003600046015701C201821993094D815E81452BD7
:1003700071F033E0883E930708F49CCF6D817E8155
:10038000615070406D837E83280E391E93CF2F817C
:1003900038858217930728F4281B390B2F83388759
:1003A000F3CFC0928401D0928501E0928601F09251
:1003B000870110938B0100938A0169847A8470927B
:1003C0008901609288012A960FB6F894DEBF0FBEAD
:1003D000CDBFDF91CF911F910F91FF90EF90DF90F4
:1003E000CF90BF90AF909F908F907F906F905F90D5
:1003F0004F903F902F9008950F931F93CF93DF93CB
:10040000EC018B01A0918C01B0918D01AB2B61F1BE
:10041000CD2B41F160EC80E090E00E948202C0E0D0
:10042000D0E0D8016C91662381F48E0121960031D1
:1004300011051CF560E281E090E00E948202AE01AD
:10044000219640315105B4F318C00F5F1F4F81E072
:1004500090E00E9482022196D8013C91632F3323C1
:10046000A1F7E3CF60E8D7CF0E94420221E030E05D
:1004700030938D0120938C01CBCFDF91CF911F91D1
:100480000F9108952FEF27BB21B32F6021BB60E0B0
:1004900070E08FE090E00E94CC0060E380E090E0AC
:1004A0000E94950260E070E085E090E00E94CC0040
:1004B00060E380E090E00E94950264E670E080E0F6
:1004C00090E00E94CC0060E380E090E00E94950202
:1004D00068E380E090E00E94820268E080E090E0C3
:1004E0000E94820261E080E090E00E94820263E06C
:1004F00080E090E00E9482026DE080E090E00E9447
:10050000820208951F93CF93DF93EC01162F80E0B2
:1005100090E00E94AD0287FDFACF612FCE010E94CC
:100520009502DF91CF911F9108952FEF27BB892B63
:1005300011F4939801C0939A9198929A68BB61E0E4
:1005400070E080E090E00E94CC00929861E070E062
:1005500080E090E00E94CC0008951F9317BA892B89
:1005600011F4939801C0939A919A929A61E070E085
:1005700080E090E00E94CC0016B3929861E070E0B9
:1005800080E090E00E94CC00812F992787FD909514
:100590001F910895109290005FE059B942E04BB965
:1005A00038E13AB926E0209395008F9A97988E9873
:1005B000969A21E030E030938301209382010895E0
:1005C000282FA0918201B0918301AB2BA9F4109246
:1005D00090007FE079B962E06BB958E15AB936E032
:1005E000309395008F9A97988E98969A41E050E0B4
:1005F00050938301409382018699FECF5D9BFCCF8F
:100600002CB90895CF93DF93EC018881882331F0D2
:1006100021960E94E00288818823D1F7DF91CF9153
:100620000895EF92FF920F931F93CF93DF93EC0106
:100630007B0197FF06C08DE20E94E002D095C19534
:10064000DF4FD7011197AC17BD0794F4CE01B70166
:100650000E94FF038B01B701C8010E9411030E9D88
:1006600090010F9D300D1E9D300D1124C21BD30B28
:10067000CF58DE4F88810E94E002DF91CF911F9119
:100680000F91FF90EF9008956F927F928F929F92BB
:10069000AF92BF92CF92DF92EF92FF920F931F9390
:1006A000CF93DF93CDB7DEB722970FB6F894DEBFB6
:1006B0000FBECDBF1FBC01E00EBD10927A007CB40E
:1006C00079826DB46A8229813A8180908A01909002
:1006D0008B01281939093695279536952795369532
:1006E00027956090880170908901620E731E709248
:1006F0008901609288016901EE24FF24D701C601B7
:1007000013E0880F991FAA1FBB1F1A95D1F78C19E8
:100710009D09AE09BF09880E991EC701B60120E4E4
:1007200030EB45E050E00E94E003E0908401F0905F
:1007300085010091860110918701E60EF71E081FC2
:10074000191FA0E4AA2EA2E4BA2EAFE0CA2ED12C23
:10075000C801B701A60195010E941204DA01C9017E
:10076000820E931E90928B0180928A01AA27BB274A
:10077000BC01CD01A60195010E94E003E61AF70A2B
:10078000080B190BE0928401F09285010093860119
:1007900010938701C30122960FB6F894DEBF0FBEF7
:1007A000CDBFDF91CF911F910F91FF90EF90DF9020
:1007B000CF90BF90AF909F908F907F906F90089553
:1007C000629FD001739FF001829FE00DF11D649F35
:1007D000E00DF11D929FF00D839FF00D749FF00DC1
:1007E000659FF00D9927729FB00DE11DF91F639F62
:1007F000B00DE11DF91FBD01CF011124089597FB34
:10080000092E07260AD077FD04D02ED006D000206E
:100810001AF4709561957F4F0895F6F7909581953C
:100820009F4F0895A1E21A2EAA1BBB1BFD010DC00C
:10083000AA1FBB1FEE1FFF1FA217B307E407F50790
:1008400020F0A21BB30BE40BF50B661F771F881F6C
:10085000991F1A9469F760957095809590959B0102
:10086000AC01BD01CF010895AA1BBB1B51E107C01C
:10087000AA1FBB1FA617B70710F0A61BB70B881F30
:10088000991F5A95A9F780959095BC01CD010895BF
:100890004B657970616420696E7465726661636529
:1008A0000A004C696E6B205043302D504333207446
:1008B0006F206B65797061642052302D52330A00CD
:1008C0004C696E6B205041302D50413320746F20A5
:1008D0006B65797061642043302D43330A00596F92
:1008E0007520747970656420613A202700313233B5
:1008F0004134353642373839432A30234400270AF9
:10090000003031323334353637383941424344458B
:0209100046009F
:00000001FF
